:10000000CAEF1BF000000000C3EF1AF00000000070
:0C001000000000000000000092EF1BF058
:08001C000AAE029E000E120064
:100024000B840BAE1DEF00F0010E036E026A016A31
:0A003400006A0A360232FF0E1200C5
:0E003E00026A016A006A086A036A000E120074
:10004C000B820BAE30EF00F00368026801680068A9
:08005C000A360232FF0E120009
:100064000CB074EF00F00CA21AEF01F00E6A000E4F
:1000740002648BEF00F0F00E0214D8A456EF00F0E7
:10008400023A01380F0B02260138F00B016E0038DA
:100094000F0B01260038F00B006E08380F0B0026FA
:1000A4000838F00B086E0E84D89002BE6FEF00F093
:1000B40008360036013602360E2A02BE6FEF00F013
:1000C40008360036013602360E2A02BE6FEF00F003
:1000D40008360036013602360E2A0E50036410EF3D
:1000E40001F0035E0BBC08AE15EF01F0D880800E62
:1000F40008640030000E002201220222D8A015EF6D
:1001040001F0023201320032034A1AEF01F015EF16
:1001140001F001C002F000C001F008C000F0086A5C
:10012400000E0E860264C2EF00F0F00E0214D8A492
:10013400AAEF00F0023A01380F0B02260138F00B47
:10014400016E00380F0B01260038F00B006E0E8490
:10015400D89002BE6FEF00F00036013602360E2A48
:1001640002BE6FEF00F00036013602360E2A02BEE0
:100174006FEF00F00036013602360E2A6FEF00F002
:1001840001C002F000C001F0006A000E0E960E8855
:100194000264EFEF00F0F00E0214D8A4DAEF00F0DE
:1001A400023A01380F0B02260138F00B016E0E845F
:1001B400D89002BE6FEF00F0013602360E2A02BE5E
:1001C4006FEF00F0013602360E2A02BE6FEF00F028
:1001D400013602360E2A6FEF00F001C002F0016A08
:1001E400000E0E8602641FEF01F0F00E0214D8A474
:1001F400FEEF00F0023A0E84D89002BE6FEF00F0DA
:1002040002360E2A02BE6FEF00F002360E2A02BE3C
:100214006FEF00F002360E2A6FEF00F0010E0C6E45
:10022400FFDE22EF01F0020E0C6EF6DE22EF01F08B
:10023400040E0C6E09DF22EF01F0080E0C6EFDDED9
:020244001200A6
:100246000A6A0350D8A40A800750D8A40A820A5022
:10025600D8B486EF01F0030AD8B43FEF01F00AB034
:100266003AEF01F006AE84EF01F082EF01F002AE44
:1002760082EF01F084EF01F00250800B0A6E029EBD
:100286000650800B069E0A18D8B450EF01F00A50AB
:10029600D8B482EF01F084EF01F00750035CD8B4C4
:1002A6005AEF01F0D8A076EF01F07CEF01F006508E
:1002B600025CD8B464EF01F0D8A076EF01F07CEFD1
:1002C60001F00550015CD8B46EEF01F0D8A076EFCE
:1002D60001F07CEF01F00450005CD8B486EF01F029
:1002E600D8B07CEF01F00A52D8B484EF01F082EF67
:1002F60001F00A52D8B482EF01F084EF01F0D88001
:0E0306001200D8901200D880D8841200120085
:10031400086A096A000E076203640FEF02F00250D4
:1003240006180A6E075003267E0ED8A0A0EF01F02F
:10033400035ED8B013EF02F0A4EF01F0035ED8A07F
:1003440017EF02F0028E068E02C00EF001C00BF011
:1003540000C00DF000500402F4CF0CF0015005026F
:10036400F4CF00F0F3CF08F00402F3500C26F4505D
:100374000822000E00220D500502F3500C26F45002
:100384000822000E002202500402F3500826F45002
:10039400002202500502016A000E0122F3500026D9
:1003A400F45001220D500602F3500826F4500022A6
:1003B400026A000E012202220B500602F3500026AC
:1003C400F4500122000E02220E500602F3500126C0
:1003D400F450022202BEF7EF01F00836003601366F
:1003E40002360306D8B417EF02F00AEF02F0D88001
:1003F400800E08640030000E002201220222D8A0E0
:100404000AEF02F0023201320032034A13EF02F023
:100414000AAE029E000E19EF02F0010E0EDE19EF75
:1004240002F0020E11DE19EF02F0040EF9DD1200E3
:100434000B800BAE26EF02F0026A0AAEFF0E026ECC
:0C044400016E006E0A360232FF0E12003C
:080450000B6A0B86FF0E12007F
:10045800025006180E6E086A096A0B6A0350076490
:100468001FEF03F006500A6E068E028E03500B6EC5
:100478000750036E000E0B646FEF02F00B50075E1F
:10048800D8B410EF03F0070E0764DEEF02F0075E42
:1004980000C008F001C000F002C001F0026A074E77
:1004A80010EF03F00764B3EF02F0075E00C008F036
:1004B80001C000F0016A074E10EF03F0076491EFE6
:1004C80002F0075E00C008F0006A074E10EF03F064
:1004D800076478EF02F00AC002F005C001F004C01A
:1004E80000F0086A3AEF04F0030E076483EF02F0A5
:1004F800075E08380F0B086E074E10EF03F0D89010
:100508000832074E10EF03F0D8900832074E10EF6C
:1005180003F0D890083210EF03F0030E0764A2EF3F
:1005280002F0075E08380F0B086E0038F00B08263B
:1005380000380F0B006E074E10EF03F0D890003212
:100548000832074E10EF03F0D89000320832074EF9
:1005580010EF03F0D8900032083210EF03F0030ECA
:100568000764CAEF02F0075E08380F0B086E003800
:10057800F00B082600380F0B006E0138F00B002630
:1005880001380F0B016E074E10EF03F0D8900132BF
:1005980000320832074E10EF03F0D89001320032D3
:1005A8000832074E10EF03F0D890013200320832BB
:1005B80010EF03F0030E0764FBEF02F0075E083844
:1005C8000F0B086E0038F00B082600380F0B006E72
:1005D8000138F00B002601380F0B016E0238F00BC2
:1005E800012602380F0B026E074E10EF03F0D89069
:1005F8000232013200320832074E10EF03F0D89071
:100608000232013200320832074E10EF03F0D89060
:100618000232013200320832096A000E0EAE04EFCF
:1006280004F0081E001E011E021E082A00220122D4
:10063800022204EF04F00750D8A425EF03F03AEFA4
:1006480004F0096A02C00AF0028E068E0750035CA5
:10065800076ED8B4F7EF03F0070E0764C5EF03F091
:10066800075E0450096E0550046E0650056E066A52
:10067800074EF7EF03F0070E07649AEF03F0075EE3
:100688000450096E0550046E056A074EF7EF03F033
:10069800070E076478EF03F0075E0450096E046ADA
:1006A800074EF7EF03F0070E07645FEF03F00AC089
:1006B80002F03AEF04F0030E07646AEF03F0075EF6
:1006C80009380F0B096E074EF7EF03F0D89009327F
:1006D800074EF7EF03F0D8900932074EF7EF03F013
:1006E800D8900932F7EF03F0030E076489EF03F09F
:1006F800075E09380F0B096E0438F00B0926043819
:100708000F0B046E074EF7EF03F0D890043209324E
:10071800074EF7EF03F0D89004320932074EF7EF8F
:1007280003F0D89004320932F7EF03F0030E0764A0
:10073800B1EF03F0075E09380F0B096E0438F00BB0
:10074800092604380F0B046E0538F00B042605380B
:100758000F0B056E074EF7EF03F0D8900532043201
:100768000932074EF7EF03F0D89005320432093208
:10077800074EF7EF03F0D890053204320932F7EF4D
:1007880003F0030E0764E2EF03F0075E09380F0B6E
:10079800096E0438F00B092604380F0B046E05386F
:1007A800F00B042605380F0B056E0638F00B0526EE
:1007B80006380F0B066E074EF7EF03F0D890063297
:1007C800053204320932074EF7EF03F0D8900632AB
:1007D800053204320932074EF7EF03F0D89006329B
:1007E800053204320932086A000E0EAE04EF04F036
:1007F800091E041E051E061E092A042205220622B9
:1008080009500826045000220550012206500222F1
:100818000EBE1BEF04F0D8A02AEF04F0023201321A
:1008280000320832033E2AEF04F034EF04F0D8B067
:100838002FEF04F0000E081E001E011E021E082ADB
:100848000022012202220A7E2FEF04F0010E0C6E14
:1008580005DC3CEF04F0020E0C6E00DC3CEF04F00B
:10086800040E0C6E26EC00F03CEF04F0000E0C6E4B
:0208780012006C
:10087A0003500718D8A451EF04F002500618D8A460
:10088A0051EF04F001500518D8A451EF04F00050BC
:0E089A000418D8B4D8841200D89412001200AA
:1008A800220E0C6E086A096A0A6A0B6A0C06D8B42A
:1008B8001FD0D8900B320A32093208320332023282
:1008C80001320032D8A0F2D70C06D8B409D00450AF
:1008D80008260550092206500A2207500B22EAD79B
:1008E800045008260550092206500A2207500B22F8
:0208F8001200EC
:1008FA000050086E0150006E0250016E0350026EE5
:10090A00036A0B6A0C6A9E0E036E0A6A02AE9AEFBB
:10091A0004F0081E001E011E021E082AD8B4002A6E
:10092A00D8B4012AD8B4022A0A8E020E0C6E32EC0E
:04093A0000F01200B7
:10093E0007012851390806E3300E285D03E3010E46
:08094E00006E01D0006A1200E6
:100956006DB409D01F0E6B14016E0150000A03E13D
:0A096600010E006E01D0006A1200BD
:1009700007012851200A09E028510D0804E3090E57
:10098000285D01E302D0006A02D0010E006E120061
:100990000C6A0E6A0250D8A4E1EF04F001C002F024
:1009A00000C001F0006A0E860250D8A4E1EF04F006
:1009B00001C002F0016A0E960E880250D8B4F3EF1F
:1009C00004F00E50035ED8A4D8A0F9EF04F0D8903C
:1009D00002BEFFEF04F0003601360236032EE8EFC8
:1009E00004F0F9EF04F0010E0C6E1FEC00F003EFC1
:1009F00005F0020E0C6E12EC00F003EF05F0040E91
:080A00000C6E0EEC00F0120078
:100A080007011D6B1E6B1E51120802E11D518E0855
:100A180008E39DDF005201E004D007011D4B1E2BA7
:100A2800F2D70701120E1E5D02E18F0E1D5D03E372
:100A38007B0E006E05D06B806BA001D0FDD7006ADD
:020A480012009A
:100A4A00A49E1DC76FFF6DA401D0FDD7A4BE01D01F
:100A5A00FDD76BBC02D0006A03D06B84020E006E15
:020A6A00120078
:100A6C001FC7F6FF20C7F7FF21C7F8FF0900F5CF16
:100A7C0000F0005218E01FC7F6FF20C7F7FF21C790
:100A8C00F8FF0900F5CF00F01DC7E1FF1EC7E2FF1C
:100A9C0000C0E6FF07011D4B1E2B010E1F27000E89
:100AAC0020232123DDD71DC7E1FF1EC7E2FFE66A25
:020ABC00120026
:100ABE000B6A0A6A096A00500402F4CF09F0F3CFF8
:100ACE0008F001500502F4CF0BF0F3CF0AF00050FE
:100ADE000502F3500926F4500A22E86A0B2201504F
:100AEE000402F3500926F4500A22E86A0B2208C0C9
:100AFE0000F009C001F00AC002F00BC003F01200B2
:0A0B0E006B826BA201D0FDD712002C
:0E0B1800ADB202D00000FCD71DC7AEFF120028
:100B2600086A080E0C6E003408360450085ED8B009
:0E0B360002D00826D89000360C2EF5D71200FB
:100B440007011F51201108E01FC7E1FF20C7E2FF82
:100B54001DC7E6FF1EC7E6FF1DC7E9FF1EC7EAFF64
:100B6400EECF00F000C023F700C028F7FFDE0052EC
:100B740003E01D4B1E2BF0D7216B000E23BFFF0E8D
:100B8400006E000E001802E12D0E231905E1010E7E
:100B9400216F1D4B1E2B0CD0000E23BFFF0E006EC9
:100BA400000E001802E12B0E231902E11D4B1E2B2F
:100BB400236B246B256B266B276B226B21B90BD01F
:100BC4001DC7E9FF1EC7EAFFEE502E0A04E1218982
:100BD4001D4B1E2B52D01DC7E9FF1EC7EAFFEECFE7
:100BE40028F7ABDE005201E149D021832351080AE2
:100BF4003FE021A901D02207232B24C700F025C7F9
:100C040001F026C702F027C703F00A0E046E000E97
:100C1400056E066E076E46DE00C024F701C025F798
:100C240002C026F703C027F7000000001DC7E9FF34
:100C34001EC7EAFF300EEE5C006E016A000E015A18
:100C4400000E01BEFF0E026E036E245100262551D4
:100C54000122265102222751032200C024F701C099
:100C640025F702C026F703C027F70000000003D0D1
:100C740021B901D0222B1D4B1E2BA0D7236B1DC7DE
:100C8400E9FF1EC7EAFFEE50650A08E01DC7E9FF49
:100C94001EC7EAFFEE50450A01E065D01D4B1E2B2E
:100CA4001DC7E9FF1EC7EAFFEE502D0A04E12187A4
:100CB4001D4B1E2B09D01DC7E9FF1EC7EAFFEE50CE
:100CC4002B0A02E11D4B1E2B1DC7E9FF1EC7EAFFBD
:100CD400EE50300A03E11D4B1E2BF6D71DC7E9FF6A
:100CE4001EC7EAFFEECF28F728DE005237E01DC703
:100CF400E9FF1EC7EAFF300EEE5C236F1D4B1E2B6F
:100D04001DC7E9FF1EC7EAFFEECF28F716DE005223
:100D140025E00A0E2303F3CF23F71DC7E9FF1EC7FF
:100D2400EAFF300EEE5C006E005023271D4B1E2B95
:100D34001DC7E9FF1EC7EAFFEECF28F7FEDD00520C
:100D44000DE00A0E2303F3CF23F71DC7E9FF1EC7E7
:100D5400EAFF300EEE5C006E0050232721A703D07B
:100D640023510008236F23512227000E201902E18A
:100D7400000E1F190AE021A308D01FC7E1FF20C7F6
:100D8400E2FF1DC7E6FF1EC7E6FF24C700F025C724
:100D940001F026C702F027C703F0ADDD00C024F739
:100DA40001C025F702C026F703C027F7046A056AC5
:100DB400066A076A24C700F025C701F026C702F0B7
:100DC40027C703F058DD010ED8A4000E006E0052B0
:100DD40005E0006A016A026A036A04D1800E2219DE
:100DE400006E800E000A005CD8B073D02251000857
:100DF400226F800E2219006E800E0A0A005C1DE329
:100E040024C700F025C701F026C702F027C703F066
:100E1400FF0E046EE60E056E5B0E066E5D0E076E2B
:100E24008AEC01F000C024F701C025F702C026F7C0
:100E340003C027F70A0E225FDCD72251000A1CE008
:100E440024C700F025C701F026C702F027C703F026
:100E5400CD0E046ECC0E056E4C0E066E7B0E076E28
:100E64008AEC01F000C024F701C025F702C026F780
:100E740003C027F72207E1D7010E046E000E056EAA
:100E8400000E066E010E076E24C700F025C701F0A0
:100E940026C702F027C703F023EC01F0010ED8B0F7
:100EA400000E006E005214E021A109D0010E006E64
:100EB400000E016E800E026E030E036E93D0010EBF
:100EC400006E000E016E000E026E010E036E8AD0DB
:100ED40072D0800E000A006E800E2219005C6BE254
:100EE4000A0E225D1DE324C700F025C701F026C7C2
:100EF40002F027C703F0F90E046E020E056E150EFC
:100F0400066EA00E076E8AEC01F000C024F701C043
:100F140025F702C026F703C027F70A0E225FE0D7A1
:100F24002251000A1CE024C700F025C701F026C79F
:100F340002F027C703F0000E046E000E056E200EAB
:100F4400066E820E076E8AEC01F000C024F701C021
:100F540025F702C026F703C027F72207E1D724C7E5
:100F640004F025C705F026C706F027C707F0FF0ED3
:100F7400006EFF0E016E7F0E026EFF0E036E23ECF9
:100F840001F0010ED8B0000E006E005214E021A151
:100F940009D0FF0E006EFF0E016EFF0E026EFF0EF3
:100FA400036E20D0FF0E006EFF0E016E7F0E026EE8
:100FB400FF0E036E17D021A10DD0000E2419006E70
:100FC400000E2519016E800E2619026E000E2719D7
:100FD400036E08D024C700F025C701F026C702F02D
:060FE40027C703F0120014
:040FEA006B84120002
:100FEE000B6A0C6A086A0350D8B47BEF08F002C093
:100FFE000AF0028E9E0E035E03AE6BEF08F0036CDA
:10100E00080E035CD8A038EF08F0036E083600C057
:10101E0008F001C000F002C001F0026A080E035C85
:10102E00D8A038EF08F0036E083600C008F001C0F3
:10103E0000F0016A080E035CD8A038EF08F0036ECA
:10104E00083600C008F0006A080E035CD8A038EF1E
:10105E0008F0036E0836086A0350D8A4D89044EFFF
:10106E0008F00350D8B444EF08F0D89002320132A1
:10107E0000320832032E3CEF08F00BBC08A055EFEF
:10108E0008F0D8A055EF08F0082AD8B4002AD8B432
:10109E00012AD8B4022A02BE7FEF08F00AAE7BEF17
:1010AE0008F0021E011E001E081E082AD8B4002ACF
:1010BE00D8B4012AD8B4022A7BEF08F0026A016A7A
:1010CE00006A086A7BEF08F00B800BAE86EF08F023
:1010DE00026A0AAE86EF08F0026E016E006E086EAE
:1010EE000A36023286EF08F00C6A000E87EF08F01F
:1010FE00010E0C6E000E1AEC02F087EF08F0FF0ED8
:10110E000250036E0150026E0050016E0850006EC8
:02111E001200BD
:101120000B6A0350D8B4D6EF08F002500A6E028E54
:101130008E0E035E03AEDAEF08F0036C080E035C5C
:10114000D8A0B5EF08F0036E013602C001F0026AC4
:10115000080E035CD8A0B5EF08F0036E0136016AF3
:101160000350D8A4D890BFEF08F00350D8B4BFEF15
:1011700008F0D89002320132032EB9EF08F00BBC10
:1011800001A0CCEF08F0D8A0CCEF08F0012AD8B429
:10119000022A02BEE9EF08F00AAEEFEF08F0021EE5
:1011A000011E012AD8B4022AEFEF08F0026A016A90
:1011B000EFEF08F00B800BAEF3EF08F0026A0AAE17
:1011C000F3EF08F0FF0E026E016E0A360232F3EF03
:1011D00008F0010E0C6E1AEC02F0F5EF08F0000EAC
:1011E0000C6EF5EF08F0FF0E0C6E0150006E025011
:0411F000016E12007A
:0811F400067E2CEC02F0120053
:1011FC000450000A12E10550000A0FE10650000AE3
:10120C000CE10750000A09E1FF0E006EFF0E016EA3
:10121C007F0E026EFF0E036EA8D0086A096A075093
:10122C00D8B4A9EF09F00350D8B4AEEF09F00250CE
:10123C0006180A6E028E068E0E6A02C008F001C0F5
:10124C000CF000C00DF004500D5E0550D8A0053C0C
:10125C000C5E0650D8A0063C085E086A0C6A0D6A43
:10126C00D8A040EF09F0D890023201320032083297
:10127C00010E0E6E0750035ED8A04DEF09F07E0EE6
:10128C000E240326D8B0B3EF09F053EF09F07E0E0D
:10129C000E240326D8A0B8EF09F0180E0B6E0D36ED
:1012AC000C3608360036013602360E360450005E17
:1012BC000550D8A0053C015E0650D8A0063C025E45
:1012CC0006340E120EA06EEF09F00D8079EF09F0C6
:1012DC00045000260550D8B0053C01260650D8B065
:1012EC00062802260D900B2E55EF09F09FEF09F002
:1012FC00D8900036013602360E360450005E05508A
:10130C00D8A0053C015E0650D8A0063C025E06340F
:10131C000E10010B0D26D8B00C2AD8B4082AD8A46C
:10132C009FEF09F008320C320D32032AD8B4B3EF18
:10133C0009F00AAE089E0850026E0C50016E0D505A
:10134C00006EBBEF09F0010E28EC02F0BBEF09F0C8
:10135C00020E1FEC00F0BBEF09F0040E26EC00F0BF
:0C136C00BBEF09F0080E12EC00F01200BC
:1013780000C008F00150006E016A026A036A0B6A35
:101388000C6A016A026A036A960E036E0A6A00AE64
:10139800D4EF09F0081E001E082AD8B4002A0A8EC5
:1013A80000C001F008C000F0086A026AC8EC04F046
:0213B800120021
:1013BA0003C704F004C705F001C702F002C703F02F
:1013CA0005C700F006C701F0010E0701055F000E10
:1013DA00065B005001100FE004C0E9FF05C0EAFFF8
:1013EA0002C0E1FF03C0E2FFEECFE6FF024A032A92
:1013FA00044A052AE5D701C700F002C701F0120026
:10140A00080E07011D6F070E1E6F05C71FF706C7D7
:10141A0020F707C721F736EC05F004EC05F0DFC624
:10142A001DF725EC05F007011D6B25EC05F0000EF4
:10143A00006E07010451005C03E103510601D25D0D
:10144A0005E2D2C603F7000E0701046F11D00701A7
:10145A000351800F1D6F1D0725EC05F017D00701FA
:10146A000351C00F1D6F1D0725EC05F00FD00ED0DC
:10147A00000E0701021902E1010E0119E8E0000E4F
:10148A00021902E1020E0119EAE0F1D787EC05F030
:10149A00DFC61DF725EC05F0400E07011D6F25EC90
:1014AA0005F003C7FEF604C7FFF605C7F6FF06C731
:1014BA00F7FF07C7F8FF0900F5CF00F0005223E055
:1014CA0005C7F6FF06C7F7FF07C7F8FF0900F5CFFC
:1014DA0000F00050800F07011D6F25EC05F0010E8A
:1014EA0007010527000E062307230601FE4BFF2BE3
:1014FA00800E006E800EFF19005C02E1FE51D25D83
:0A150A0001E201D0D2D76CDD12001F
:1015140004C700F0016A026A036AFF0E0016000E97
:10152400011600C0FEF601C0FFF67F0E005C026EDD
:10153400000E0158036E02C0FEF603C0FFF6800ED3
:101544000318006E800E005C02E1000E025C22E2D1
:10155400046A056A066A076A01C700F002C701F057
:1015640003C702F004C703F023EC01F0010ED8B066
:10157400000E006E005209E0000E006E000E016EB7
:10158400800E026E7F0E036E5CD0006A016A026AEE
:10159400036A57D0000E006E0601FF51005C02E1A1
:1015A400FE51180809E201C700F002C701F003C7A1
:1015B40002F004C703F045D001C700F002C701F0F0
:1015C40003C702F004C703F010DD7DEC04F000C093
:1015D40005F701C006F702C007F703C008F700C00B
:1015E40004F001C005F002C006F003C007F001C713
:1015F40000F002C701F003C702F004C703F023ECB4
:1016040001F0010ED8B0000E006E005212E0000E80
:10161400046E000E056E000E066E7F0E076E05C783
:1016240000F006C701F007C702F008C703F0E0DDC9
:1016340008D005C700F006C701F007C702F008C7C5
:0416440003F012009D
:1016480004EC05F0DFC61DF725EC05F007011D6B5E
:1016580025EC05F0020E07011D6F25EC05F00DD0F5
:10166800800E07011D6F25EC05F015D0C00E07018F
:101678001D6F25EC05F00FD00ED0000E0601FF19E6
:1016880002E1010EFE19ECE0000EFF1902E1020E64
:10169800FE19ECE0F1D787EC05F0DFC61DF725EC65
:1016A80005F0400E07011D6F25EC05F00701016BE1
:1016B800026B800E0219006E800E005C04E10601C8
:1016C800D2510701015D08E2A00E1D6F25EC05F05F
:1016D8000701014B022BEDD787EC05F0DFC61DF79C
:1016E80025EC05F007011D6B25EC05F00DD0800EEB
:1016F80007011D6F25EC05F015D0C00E07011D6F01
:1017080025EC05F00FD00ED0000E0601FF1902E1FE
:10171800010EFE19ECE0000EFF1902E1020EFE199F
:08172800ECE0F1D75EDC1200D9
:1017300004EC05F0DFC61DF725EC05F007011D6B75
:1017400025EC05F0000E006E07010451005C03E17A
:1017500003510601D25D05E2D2C603F7000E070170
:10176000046F11D007010351800F1D6F1D0725EC79
:1017700005F017D007010351C00F1D6F1D0725ECA1
:1017800005F00FD00ED0000E0701021902E1010E84
:101790000119E8E0000E021902E1020E0119EAE067
:1017A000F1D787EC05F0DFC61DF725EC05F0400EFC
:1017B00007011D6F25EC05F003C7FEF604C7FFF611
:1017C00005C7E9FF06C7EAFFEE521BE005C7D9FFD0
:1017D00006C7DAFFDE50800F07011D6F25EC05F00C
:1017E0000701054B062B0601FE4BFF2B800E006EFA
:1017F000800EFF19005C02E1FE51D25D01E201D0D2
:08180000DFD7F5EC07F0120040
:0E180800A8B202D00000FCD7FEC6A9FF120055
:1018160007010751000806E3070E0601FE6F000EDA
:10182600FF6F13D007010751160805E2170E086F60
:10183600000E096F06D00751010F086F096B000EE5
:10184600092308C7FEF609C7FFF60701FEC610F70B
:10185600FFC611F70A6B0B6B046A056A066A076A0C
:1018660001C700F002C701F003C702F004C703F086
:1018760023EC01F0010ED8B0000E006E005209E014
:1018860005C7E1FF06C7E2FF2D0EE66E054B062BE8
:10189600037F01C704F002C705F003C706F004C7BB
:1018A60007F0006A016A026A036A23EC01F0010E7E
:1018B600D8B0000E006E005237E0000E046E000E27
:1018C600056E000E066E7F0E076E01C700F002C79A
:1018D60001F003C702F004C703F023EC01F0010E88
:1018E600D8B0000E006E00521FE001C700F002C71C
:1018F60001F003C702F004C703F0000E046E000EE9
:10190600056E200E066E820E076E8AEC01F000C090
:1019160001F701C002F702C003F703C004F7010E86
:101926000A5F000E0B5BC9D7000E046E000E056E33
:10193600200E066E820E076E01C700F002C701F088
:1019460003C702F004C703F023EC01F0000ED8B081
:10195600010E006E00521DE0000E046E000E056EB4
:10196600200E066E820E076E01C700F002C701F058
:1019760003C702F004C703F03EDC00C001F701C054
:1019860002F702C003F703C004F707010A4B0B2B4B
:10199600CBD70A5110270B511123010E0C6F000EE5
:1019A6000D6F000E126F000E136F000E146F7F0E78
:1019B600156F800E0D19006E800E1119005C02E184
:1019C60010510C5D1DE2000E046E000E056E200E19
:1019D600066E820E076E12C700F013C701F014C719
:1019E60002F015C703F007DC00C012F701C013F7B9
:1019F60002C014F703C015F707010C4B0D2BD9D7FE
:101A0600000E046E000E056E000E066E800E076E4A
:101A160012C700F013C701F014C702F015C703F090
:101A2600FEEC08F001C704F002C705F003C706F094
:101A360004C707F02CEC02F000C001F701C002F762
:101A460002C003F703C004F7000E046E000E056E15
:101A5600200E066E820E076E23EC01F0000ED8B043
:101A6600010E006E00520BE0000E0701016F000E22
:101A7600026F000E036F7F0E046F0A4B0B2B0701DC
:101A8600800E0B19006E800E005C02E1000E0A5DEE
:101A960038E205C7E1FF06C7E2FF300EE66E054BEA
:101AA600062B05C7E1FF06C7E2FF2E0EE66E054BC5
:101AB600062B800E1119006E800E005C02E1000EEE
:101AC600105D04E210510A5F11510B5BFF0E0C6FA3
:101AD600FF0E0D6F800E0B19006E800E0D19005C47
:101AE60002E10C510A5D0DE205C7E1FF06C7E2FF00
:101AF600300EE66E054B062B010E0C5F000E0D5BDD
:101B0600E9D70C6B0D6B800E0D19006E800E111946
:101B1600005C02E110510C5D62E201C700F002C7F1
:101B260001F003C702F004C703F090EC08F000C010
:101B36000EF701C00FF7300E002605C7E1FF06C7F6
:101B4600E2FF00C0E6FF054B062B0D510B1902E123
:101B56000A510C1908E105C7E1FF06C7E2FF2E0E80
:101B6600E66E054B062B0EC700F00FC701F001DC31
:101B760000C012F701C013F702C014F703C015F72F
:101B860000C004F001C005F002C006F003C007F073
:101B960001C700F002C701F003C702F004C703F053
:101BA600FAEC08F000C001F701C002F702C003F723
:101BB60003C004F7000E046E000E056E200E066EBE
:101BC600820E076E8AEC01F000C001F701C002F731
:101BD60002C003F703C004F70C4B0D2B94D705C7BF
:0A1BE600E1FF06C7E2FFE66A120005
:101BF0000601FE6B030EFE5D0CE2FE51070102259D
:101C0000E16E000E0321E26E200EE66E0601FE2B51
:101C1000F1D7FE5107010225E16E000E0321E26EAD
:101C2000E66A0601FE07FE51070102250601FF6F65
:101C3000000E07010321006F0A0E046E01C700F0B9
:101C400093EC05F008C000F0300E0026FFC6E1FF5F
:101C500000C7E2FF00C0E6FF0A0E046E01C700F0F5
:101C600093EC05F000C001F70050000A01E103D039
:081C70000601FE07D8D712009F
:101C78000D0E07011D6F8CEC05F00A0E07011D6F94
:061C88008CEC05F01200D7
:101C8E0001C7F6FF02C7F7FF03C7F8FF0900F5CF3C
:101C9E0000F0005212E001C7F6FF02C7F7FF03C7BC
:101CAE00F8FF0900F5CF1DF78CEC05F0010E0701CA
:0C1CBE000127000E02230323E3D71200CD
:101CCA00086A096A100E0C6E013408360936045087
:101CDA00085E0550D8A0053C095ED8B007D004506C
:101CEA0008260550D8B0053C0926D890003601369A
:061CFA000C2EEAD71200D7
:101D0000FEC6E9FFFFC6EAFFEECF01F7000E0701AE
:101D1000026F000E026F000E021902E1200E01197F
:101D200007E0000E021902E1090E011901E004D0DA
:101D30000601FE4BFF2BE4D70701036B046B056B19
:101D4000066B000E021902E12D0E011906E1054B8A
:101D5000062B0601FE4BFF2B0AD0000E07010219CD
:101D600002E12B0E011903E10601FE4BFF2BFEC61B
:101D7000E9FFFFC6EAFFEECF01F7000E0701026F91
:101D8000000E026F01C728F79FEC04F000521AE022
:101D900003C700F004C701F00A0E046E000E056EC2
:101DA0005FEC05F0300E015D026E000E0259036E0D
:101DB00002500024036F03500120046F0601FE4B04
:101DC000FF2BD5D707010551061108E00351000884
:101DD000006E04C701F0000E015604D003C700F0E6
:061DE00004C701F012002F
:101DE60001C704F002C705F004C002F005C003F005
:101DF600044A052A03C700F004C701F00701034B94
:101E0600042B00C0E9FF01C0EAFF02C0E1FF03C0E6
:101E1600E2FFEECFE6FF02C0E9FF03C0EAFFEE52A3
:0E1E260001E0E2D701C700F002C701F0120090
:101E3400A49E6B86A4BE01D0FDD76FCF01F006012E
:101E4400FE51000A02E16B8A01D06B9AA49E6B8852
:0C1E5400A4BE01D0FDD701C000F01200B8
:101E600001C704F002C705F004C0E9FF05C0EAFF9E
:101E7000EE5203E0044A052AF7D704C002F005C079
:101E800003F0044A052A03C700F004C701F0070164
:101E9000034B042B00C0E9FF01C0EAFF02C0E1FFD1
:101EA00003C0E2FFEECFE6FF02C0E9FF03C0EAFF96
:101EB000EE5201E0E2D701C700F002C701F01200C4
:101EC0000701016BFEC6E9FFFFC6EAFFEECF00F790
:101ED00007010051000A10E000C71DF78CEC05F067
:101EE0000701012B01510601FE25E96E000EFF21BD
:0A1EF000EA6EEECF00F7ECD7120007
:101EFA00FEC602F0FFC603F002C000F003C001F004
:101F0A00024A032A00C0E9FF01C0EAFFEE5201E0DB
:101F1A00F3D70601FE51025C006EFF510358016EB1
:0A1F2A00010E005E000E015A1200C5
:101F3400FEC61DF7FFC61EF707011F6B206BA2EC40
:041F440005F0120092
:101F48000601F46BF56B1F0E0B6E710E0C6E1E0EF8
:101F58000D6E0D2EFED70C2EFCD70B2EFAD70000D7
:101F680004EC05F0DFC61DF725EC05F000C0F2F61D
:101F7800000E0601F36F000EF31902E1000EF219CC
:101F880005E0F4C600F0F5C601F0E6D0F44BF52BF9
:101F98000D0E0B6E2D0E0C6ED70E0D6E0D2EFED780
:101FA8000C2EFCD70B2EFAD70000000007011D6B82
:101FB80025EC05F000C0F2F6000E0601F36F800E66
:101FC800006E800EF319005C02E1F251000805E290
:101FD800F4C600F0F5C601F0BFD0F44BF52B240E83
:101FE80007011D6F25EC05F00C0E07011D6F25EC90
:101FF80005F0060E07011D6F25EC05F0250E0701FB
:102008001D6F25EC05F0060E07011D6F25EC05F088
:10201800110E07011D6F25EC05F0420E07011D6F1B
:1020280025EC05F0960E07011D6F25EC05F0240E32
:1020380007011D6F25EC05F000C0F2F6000E060141
:10204800F36F800E006E800EF319005C02E1F2510E
:10205800000805E2F4C600F0F5C601F07DD0F44BA7
:10206800F52B0C0E07011D6F25EC05F000C0F2F6EC
:10207800000E0601F36F800E006E800EF319005CEF
:1020880002E1F251000805E2F4C600F0F5C601F0DD
:1020980063D0F44BF52B060E07011D6F25EC05F0F8
:1020A80000C0F2F6000E0601F36F800E006E800E7F
:1020B800F319005C02E1F251000805E2F4C600F0F1
:1020C800F5C601F049D0F44BF52B020E07011D6F40
:1020D80025EC05F000C0F2F6000E0601F36F800E45
:1020E800006E800EF319005C02E1F251000805E26F
:1020F800F4C600F0F5C601F02FD0F44BF52B010E15
:1021080007011D6F25EC05F000C0F2F6000E060170
:10211800F36F800E006E800EF319005C02E1F2513D
:10212800000805E2F4C600F0F5C601F015D0070E68
:102138000B6E170E0C6E6A0E0D6E0D2EFED70C2E42
:10214800FCD70B2EFAD70000F5EC07F0F44BF52B73
:0A215800F4C600F0F5C601F0120015
:10216200180E0601E06F0B0EE16F1D0EE26F070EF7
:10217200E36FFF0EDB6FFF0EDC6F000EDD6F000EF4
:10218200DE6FFF0ED36FFF0ED46F000ED56F000E01
:10219200D66FFF0ED76FFF0ED86F000ED96F000EED
:1021A200DA6FAD8A900EAC6E948E949C9EAA03D088
:0821B200AFCF00F0FBD71200D3
:1021BA00FF0E926E020EC16EFF0EC26EFF0E936E7E
:1021CA00FF0E956EFF0E946EFF0E986E959C958E7F
:1021DA009986959896988C988D98938093821200F8
:1021EA000900F5CFE6FF0006FBE10106F9E112005E
:1021FA00080E0601E06F180EE16FFE0EE26F060E82
:10220A00E36FFF0EDB6FFF0EDC6F000EDD6F000E5B
:10221A00DE6FFF0ED36FFF0ED46F000ED56F000E68
:10222A00D66FFF0ED76FFF0ED86F000ED96F000E54
:10223A00DA6FA88A900E9C6E98849892A4AA03D00A
:08224A00AACF00F0FBD712003F
:102252002B0E0701016F4B0E026F000E036F16DD8E
:10226200F2C601F7F40E0701026F060E036FBFDC20
:10227200F40E0601FE6F060EFF6F21DED90E070176
:10228200016F4B0E026F000E036F00DDD00E0701CF
:10229200016F4B0E026F000E036FF8DC04EC05F0C9
:1022A200F2C61DF725EC05F000C0F3F60050000A57
:1022B2000BE0490E0701016F4B0E026F000E036F18
:1022C200E5DC0601F36B0BD0AB0E0701016F4B0E81
:1022D200026F000E036FDADC010E0601F36FF5ECFC
:0A22E20007F0C9DCF3C600F012009B
:1022EC00150E7B6EA00E7A6E0501816B826B799256
:1022FC00798A7988799C79967994798E7990A29259
:06230C00A192A092120054
:10231200959A959C8C9A8C9C958A958C6D9E6D9CB9
:06232200380E6C6E120083
:10232800020E0601FE6F000EFF6F24EC0BF0010E8B
:0E2338000601FE6F000EFF6F24EC0BF012008A
:102346000601F56BF2C6E9FFF3C6EAFFEECFF4F637
:10235600F451000A0FE0F4C6FEF604EC0CF0060198
:10236600F52BF551F225E96E000EF321EA6EEECF5C
:06237600F4F6EED71200A0
:10237C00440E0601FE6F000EFF6F9CDDE90E070197
:10238C00016F4B0E026F000E036F7BDC870E060194
:10239C00FE6F040EFF6FC8DD00C0E6F601C0E7F665
:1023AC0002C0E8F603C0E9F6000E046E000E056EDE
:1023BC00480E066E850E076EFEEC08F000C05EF54A
:1023CC0001C05FF502C060F503C061F500C001F704
:1023DC0001C002F702C003F703C004F78AEC0AF04D
:1023EC0000C0F2F601C0F3F602C0F4F603C0F5F635
:1023FC00F2C65EF5F3C65FF5F4C660F5F5C661F599
:10240C00000E046E000E056E480E066E850E076EED
:10241C00E6C600F0E7C601F0E8C602F0E9C603F034
:10242C00FEEC08F0F2C604F0F3C605F0F4C606F0B4
:10243C00F5C607F0FAEC08F000C058F501C059F5E4
:10244C0002C05AF503C05BF5000E046E000E056E5B
:10245C00480E066E850E076E8AEC01F0000E046EB7
:10246C00000E056E700E066E840E076EFEEC08F004
:10247C00F2C604F0F3C605F0F4C606F0F5C607F094
:10248C002CEC02F000C0E6F601C0E7F602C0E8F65C
:10249C0003C0E9F606018B51530A1AE1E6C600F0B7
:1024AC00E7C601F0E8C602F0E9C603F0000E046EC0
:1024BC00000E056E800E066E7F0E076E8AEC01F024
:1024CC0000C0E6F601C0E7F602C0E8F603C0E9F684
:1024DC00E6C601F7E7C602F7E8C603F7E9C604F754
:1024EC009C0E0701056F060E066F060E076F0BECB0
:1024FC000CF005015C6B5D6B000E5D5D02E11F0E67
:10250C005C5D0BE2550E5C25E16E000E5D21E26E0A
:10251C00200EE66E5C4B5D2BEFD7556A550E07010E
:10252C00016F000E026F9C0E036F060E046F55DCDC
:10253C00550E016F000E026F1F0E036F000E046F1D
:10254C0089DC9C0E0601FE6F060EFF6FB3DC200EBD
:10255C0007011D6F8CEC05F08BC61DF78CEC05F09C
:10256C00C70E0701016F4B0E026F000E036F47EC95
:10257C000EF07C0E0601FE6F040EFF6FD5DC00C062
:10258C00EAF601C0EBF602C0ECF603C0EDF6000E65
:10259C00046E000E056E480E066E850E076EFEEC80
:1025AC0008F000C05EF501C05FF502C060F503C025
:1025BC0061F500C001F701C002F702C003F703C0C8
:1025CC0004F78AEC0AF000C0F2F601C0F3F602C080
:1025DC00F4F603C0F5F6F2C65EF5F3C65FF5F4C685
:1025EC0060F5F5C661F5000E046E000E056E480E22
:1025FC00066E850E076EEAC600F0EBC601F0ECC65F
:10260C0002F0EDC603F0FEEC08F0F2C604F0F3C6DF
:10261C0005F0F4C606F0F5C607F0FAEC08F000C0B9
:10262C0058F501C059F502C05AF503C05BF5000E10
:10263C00046E000E056E480E066E850E076E8AEC53
:10264C0001F0000E046E000E056E700E066E840E08
:10265C00076EFEEC08F0F2C604F0F3C605F0F4C603
:10266C0006F0F5C607F02CEC02F000C0EAF601C04B
:10267C00EBF602C0ECF603C0EDF60601EE51570A7C
:10268C001AE1EAC600F0EBC601F0ECC602F0EDC6AA
:10269C0003F0000E046E000E056E800E066E7F0EAB
:1026AC00076E8AEC01F000C0EAF601C0EBF602C03E
:1026BC00ECF603C0EDF6EAC601F7EBC602F7ECC682
:1026CC0003F7EDC604F79C0E0701056F060E066FA7
:1026DC00060E076F0BEC0CF0550E016F000E026F1F
:1026EC009C0E036F060E046F30EC0FF0550E016F4D
:1026FC00000E026F1D0E036F000E046F30EC0FF016
:10270C009C0E0601FE6F060EFF6F60EC0FF0200EA4
:10271C0007011D6F8CEC05F0EEC61DF78CEC05F077
:10272C007E0E0701016F4B0E026F000E036F47EC1C
:10273C000EF08C0E0601FE6F060EFF6F9AEC0FF07A
:10274C0000C04FF001C050F002C051F003C052F075
:10275C0000C001F701C002F702C003F703C004F781
:10276C009C0E056F060E066F010E076F0BEC0CF03E
:10277C00550E016F000E026F9C0E036F060E046F58
:10278C0030EC0FF09C0E0601FE6F060EFF6F60EC36
:10279C000FF0200E00016D6F746B960E0701016F28
:1027AC004B0E026F000E036F47EC0EF0620E06012B
:1027BC00FE6F050EFF6F60EC0FF08A0E0701016FC4
:1027CC004B0E026F000E036F47EC0EF0660E060107
:1027DC00FE6F050EFF6F60EC0FF0A10E0701016F8D
:1027EC004B0E026F000E036F47EC0EF057C51DF732
:1027FC008CEC05F0200E0001746F3CEC0EF0120016
:10280C000601F46BF56B010EF86F000EF96F970E65
:10281C00FE6F040EFF6F7DEC0FF000C0F6F601C0EA
:10282C00F7F6070EF26F000EF36F800EF319006EC1
:10283C00800EF719005C02E1F651F25DD8B089D137
:10284C0046D1970EF225E96E040EF321EA6EEE5096
:10285C002C0A0EE1C40EF425E16E060EF521E26E93
:10286C00E66AF46BF56B020EF86F000EF96F6ED121
:10287C00C40EF425E16E060EF521E26E970EF225DC
:10288C00E96E040EF321EA6EEECFE6FFF44BF52B66
:10289C005DD1970EF225E96E040EF321EA6EEE502F
:1028AC002C0A0EE17C0EF425E16E040EF521E26E8D
:1028BC00E66AF46BF56B030EF86F000EF96F46D1F8
:1028CC007C0EF425E16E040EF521E26E970EF225D6
:1028DC00E96E040EF321EA6EEECFE6FFF44BF52B16
:1028EC0035D1970EF225E96E040EF321EA6EEE5007
:1028FC002C0A07E1F46BF56B040EF86F000EF96F00
:10290C0025D1970EF225E96E040EF321EA6EEECF77
:10291C008BF6F44BF52B1AD1970EF225E96E040EBB
:10292C00F321EA6EEE502C0A0EE1870EF425E16ECF
:10293C00040EF521E26EE66AF46BF56B050EF86F8A
:10294C00000EF96F03D1870EF425E16E040EF5210C
:10295C00E26E970EF225E96E040EF321EA6EEECFCD
:10296C00E6FFF44BF52BF2D0970EF225E96E040E30
:10297C00F321EA6EEE502C0A07E1F46BF56B060EB0
:10298C00F86F000EF96FE2D0970EF225E96E040E87
:10299C00F321EA6EEECFEEF6F44BF52BD7D0970E73
:1029AC00F225E96E040EF321EA6EEE502C0A07E1D3
:1029BC00F46BF56B070EF86F000EF96FC7D0970E1E
:1029CC00F225E96E040EF321EA6EEECF57F5F44BC7
:1029DC00F52BBCD0970EF225E96E040EF321EA6EAE
:1029EC00EE502C0A0EE1620EF425E16E050EF52177
:1029FC00E26EE66AF46BF56B080EF86F000EF96F79
:102A0C00A5D0620EF425E16E050EF521E26E970E4F
:102A1C00F225E96E040EF321EA6EEECFE6FFF44BDD
:102A2C00F52B94D0970EF225E96E040EF321EA6E85
:102A3C00EE502C0A0EE1660EF425E16E050EF52122
:102A4C00E26EE66AF46BF56B090EF86F000EF96F27
:102A5C007DD0660EF425E16E050EF521E26E970E23
:102A6C00F225E96E040EF321EA6EEECFE6FFF44B8D
:102A7C00F52B6CD0970EF225E96E040EF321EA6E5D
:102A8C00EE502C0A0EE18C0EF425E16E060EF521AB
:102A9C00E26EE66AF46BF56B0A0EF86F000EF96FD6
:102AAC0055D08C0EF425E16E060EF521E26E970ED4
:102ABC00F225E96E040EF321EA6EEECFE6FFF44B3D
:102ACC00F52B44D0F6C6F2F6F7C6F3F63FD0000E5F
:102ADC00F91902E1010EF819D8B4B3D6000EF919A0
:102AEC0002E1020EF819D8B4D4D6000EF91902E19D
:102AFC00030EF819D8B4F5D6000EF91902E1040E3C
:102B0C00F819D8B409D7000EF91902E1050EF81915
:102B1C00D8B42AD7000EF91902E1060EF819D8B468
:102B2C003ED7000EF91902E1070EF819D8B452D7A6
:102B3C00000EF91902E1080EF819D8B473D7000E7B
:102B4C00F91902E1090EF81995E0BCD7F24BF32BF9
:0C2B5C006CD6F8C600F0F9C601F01200BB
:102B6800F2C604F0F3C605F00601F651F71124E0A9
:102B7800010EF65F000EF75B04C002F005C003F01B
:102B8800044A052AF4C600F0F5C601F0F44BF52B0B
:102B980000C0E9FF01C0EAFF02C0E1FF03C0E2FF95
:102BA800EECFE6FF02C0E9FF03C0EAFFEECF00F078
:102BB800005201E101D0D8D7F6C600F0F7C601F0FF
:102BC800010EF65F000EF75B0050011008E004C02C
:102BD800E1FF05C0E2FFE66A044A052AEDD7F2C61E
:082BE80000F0F3C601F0120039
:102BF000010E0601FE6F000EFF6F24EC0BF09C0E21
:102C000007011D6F060E1E6FE70E1F6F4A0E206F25
:102C1000000E216F36EC05F08C0E0601FE6F060EDD
:102C2000FF6F7DEC0FF000500608026E01C003F04C
:102C3000000E035602C0F2F603C0F3F6800E03182E
:102C4000006E800E005C02E1000E025C02E2F26B9C
:102C5000F36BF251A7080701016FF3C602F7060EE6
:102C600002578C0E036F060E046FF3EC0EF06D0E20
:102C70000601AB6F010E0701016F000E026F010E1E
:102C8000036F000E046F9C0E056F060E066F98EC26
:102C90000BF0020E0601FE6F000EFF6F24EC0BF02E
:102CA0009C0E07011D6F060E1E6F720E1F6F4B0EDE
:102CB000206F000E216F36EC05F0F40E0701016F56
:102CC000060E026FC40E036F060E046F020E056F30
:102CD000000E066FDDEC09F0F40E0601FE6F060E25
:102CE000FF6F80EC0EF0010E0024026E000E01203A
:102CF000036E02C0F8F603C0F9F6800E006E800E77
:102D00000318005C02E10250170803E20601F86BA9
:102D1000F96B0601D0C600F0D1C601F0000E026EBC
:102D2000036E100E046E270E056E000E066E000E6A
:102D3000076E54EC04F000C0FAF601C0FBF602C0C6
:102D4000FCF603C0FDF6E4C600F0E5C601F0000E97
:102D5000026E036E640E046E000E056E066E076E44
:102D600054EC04F00050FA25046E0150FB21056E6E
:102D70000250FC21066E0350FD21076EF0C600F0E4
:102D8000F1C601F0000E026E036E005004260150E1
:102D90000522025006220350072204C03CF005C061
:102DA0003DF006C03EF007C03FF0800E0718006EF1
:102DB000800E000A005C08E1020E065C05E1720E5E
:102DC000055C02E1470E045C12E3800E3F18006EC2
:102DD000800E000A005C08E1020E3E5C05E1750E03
:102DE0003D5C02E1060E3C5C02E20601EF8F800EC4
:102DF0003F18006E800E000A005C08E1020E3E5C87
:102E000005E1750E3D5C02E1060E3C5C12E3800EAE
:102E10003F18006E800E000A005C08E11A0E3E5C4E
:102E200005E1DC0E3D5C02E1460E3C5C02E206017F
:102E3000EF9F800E3F18006E800E000A005C08E1D4
:102E4000020E3E5C05E1990E3D5C02E1560E3C5CD3
:102E500012E3800E3F18006E800E000A005C08E14D
:102E6000020E3E5C05E19C0E3D5C02E1150E3C5CF1
:102E700002E20601EF8F0601EFAF02D0F84BF92B0B
:102E8000800E006E800EF919005C02E1F8511708FF
:102E900002E2F86BF96BC40EFE6F060EFF6F7DEC5D
:102EA0000FF000C0F2F601C0F3F6F8C601F7F40E19
:102EB0000701026F060E036FF8EC0DF09C0E070180
:102EC000016F060E026FF50E036F060E046F020E01
:102ED000056F000E066FDDEC09F09F0E016F060E08
:102EE000026FC60E036F060E046F020E056F000E12
:102EF000066FDDEC09F0A20E016F060E026FC80E20
:102F0000036F060E046F020E056F000E066FDDECF8
:102F100009F00601AC6B440E0701016F000E026F51
:102F20009C0E036F060E046FF3EC0EF0020E016FA1
:102F3000000E026F010E036F000E046F100E056F7E
:102F40004C0E066F000E076F05EC0AF0020E07012B
:102F5000016F000E026F070E036F000E046F9C0ED0
:102F6000056F060E066F98EC0BF05C0E0B6E510EA3
:102F70000C6E600E0D6E0D2EFED70C2EFCD70B2E98
:102F8000FAD700009C0E07011D6F060E1E6FB40ECF
:102F90001F6F4A0E206F000E216F36EC05F0E6C65B
:102FA00001F7E7C602F7E8C603F7E9C604F7A10E82
:102FB0000701056F060E066F060E076F0BEC0CF08F
:102FC0009C0E0601FE6F060EFF6F7DEC0FF0800E6B
:102FD0000118026E800E025C02E1100E005C0CE231
:102FE0009C0E0701016F060E026F420E036F000E6A
:102FF000046F30EC0FF0E4D7EEC6ABF60601AC6B15
:10300000010E0701016F000E026F010E036F000E2B
:10301000046F9C0E056F060E066F98EC0BF09C0E6D
:1030200007011D6F060E1E6FD60E1F6F4A0E206F12
:10303000000E216F36EC05F0EAC601F7EBC602F789
:10304000ECC603F7EDC604F7A10E0701056F060EE7
:10305000066F060E076F0BEC0CF09C0E0601FE6F60
:10306000060EFF6F7DEC0FF0800E0118026E800ED1
:10307000025C02E1100E005C0CE29C0E0701016F85
:10308000060E026F400E036F000E046F30EC0FF05F
:10309000E4D78BC6ABF60601AC6B020E0701016FDD
:1030A000000E026F010E036F000E046F9C0E056F81
:1030B000060E066F98EC0BF05C0E0B6E510E0C6E4C
:1030C000600E0D6E0D2EFED70C2EFCD70B2EFAD7F0
:0430D00000001200EA
:1030D40005017E6B7F6BF2AE03D0010E0601F66F25
:1030E400F29E090E006EF2C603F0F3C604F000501F
:1030F40005E004320332049EFF0FFAD703C000F048
:1031040004C001F000360090013600C0F4F601C09E
:10311400F5F60050A00F0501806F070E006EF2C691
:10312400F4F6F3C6F5F6005006E00601F437F49120
:10313400F537FF0FF9D704EC05F080C51DF725EC32
:1031440005F0F5C61DF725EC05F0F4C61DF725ECD2
:1031540005F00050000803E205017E4B7F2B0601B9
:10316400F46BF56B000EF55D02E17F0EF45D1CE27D
:10317400860EF425E96E050EF521EA6EEECF1DF7F5
:1031840025EC05F00050000803E205017E4B7F2B7F
:103194004E0E0C6EEB0E0D6E0D2EFED70C2EFCD7C4
:1031A4000601F44BF52BDED7F5EC07F0ABEC04F09D
:0C31B4000601F651010AD8B4F28E120098
:1031C00005017E6B7F6BF2AE03D0010E0601F66F38
:1031D000F29E090E006EF2C603F0F3C604F0005032
:1031E00005E004320332049EFF0FFAD703C000F05B
:1031F00004C001F000360090013600C0F4F601C0B2
:10320000F5F60050A00F0501806F070E006EF2C6A4
:10321000F4F6F3C6F5F6005006E00601F437F49133
:10322000F537FF0FF9D704EC05F080C51DF725EC45
:1032300005F0F5C61DF725EC05F0F4C61DF725ECE5
:1032400005F00050000803E205017E4B7F2B87EC60
:1032500005F005018051010F07011D6F25EC05F0F8
:10326000ABEC04F00601F46BF56B000EF55D02E1CA
:103270007E0EF45D14E2860EF425F76F050EF5213F
:10328000F86F010EFE6F1AEC0FF0F7C6E1FFF8C6FB
:10329000E2FF00C0E6FF0601F44BF52BE6D7860EF1
:1032A000F425F76F050EF521F86FFE6B1AEC0FF0A1
:1032B000F7C6E1FFF8C6E2FF00C0E6FFF5EC07F055
:1032C000ABEC04F0040E0B6E0C0E0C6E330E0D6E98
:1032D0000D2EFED70C2EFCD70B2EFAD700000000C7
:0C32E0000601F651010AD8B4F28E12006B
:1032EC000601F66B050EF65D0AE2F651F425E16E69
:1032FC00000EF521E26E200EE66EF62BF3D7F6519A
:10330C00F425E16E000EF521E26EE66AF607F65141
:10331C00F425F76F000EF521F86F0A0E046E000EFF
:10332C00056EF2C600F0F3C601F065EC0EF008C0B5
:10333C0000F009C001F0300E0026F7C6E1FFF8C618
:10334C00E2FF00C0E6FF0A0E046E000E056EF2C628
:10335C0000F0F3C601F065EC0EF000C0F2F601C00F
:10336C00F3F6000E011802E1000E001801E102D084
:06337C00F607CDD7120098
:10338200FF0E05017A6FFF0E7B6FFF0E7C6FFF0E43
:0E3392007D6FC26A070EC16EC18EC28012002E
:1033A000536A546A020E545C02E1000E535C0AE256
:1033B000750E5324E16E000E5420E26EE66A534A05
:1033C000542AF0D70401796B7A6B536A546A9EAA27
:1033D00002D0AFCF7BF47B6B776B786BA08A120047
:1033E0000201756B766B020E765D02E1000E755D73
:1033F0000AE2770E7525E16E020E7621E26EE66A2C
:10340000754B762BF0D705016E6B6F6B0201756BF8
:10341000766BA4AA02D0AACF83F50501836B846BD7
:06342000856BA38A120077
:10342600210E07011D6F000E1E6FB50E1F6F4B0E8E
:10343600206F000E216F36EC05F02CC521F02DC54E
:1034460022F02EC524F02FC525F030C527F031C552
:1034560028F0296A210E0601FE6F000EFF6F60EC50
:103466000FF0200E07011D6F8CEC05F0200E0701F2
:103476001D6F8CEC05F0300E05012C5D006E016AA7
:10348600000E015A0A0E046E000E056E5FEC05F082
:103496002D5100240601F06F000E0120F16F300E51
:1034A600F05F000EF15B300E05012E5D006E016AC5
:1034B600000E015A0A0E046E000E056E5FEC05F052
:1034C6002F5100240601E46F000E0120E56F300E37
:1034D600E45F000EE55B300E0501305D006E016AAB
:1034E600000E015A0A0E046E000E056E5FEC05F022
:1034F600315100240601D06F000E0120D16F300E2D
:08350600D05F000ED15B120042
:10350E00F6C600F00601F607005228E0F2C6E9FF03
:10351E00F3C6EAFFEE50000A0CE0F2C6E9FFF3C66E
:10352E00EAFFF4C6D9FFF5C6DAFFEE50DE1801E168
:10353E000FD0F2C6E9FFF3C6EAFFF4C6D9FFF5C60F
:10354E00DAFFDE50EE5C006E016A000E015A08D002
:10355E000601F24BF32BF44BF52BD2D7006A016A1E
:02356E00120049
:10357000150E7B6EA00E7A6E0501816B826BA19297
:06358000A0827980120018
:1035860000C01AF0E1CF1BF0E2CF1CF09EAA45D096
:103596009DAA43D0ACA203D0AC98AC88AC92ACA4A4
:1035A60002D0AFCF7BF4AFCF7BF404017B510D0A81
:1035B60007E0020E545C02E1000E535C01E21FD0EC
:1035C6000401010E776F000E786F020E545C02E163
:1035D600000E535C04E3020E776F000E786FA09A1C
:1035E600750E5324E16E000E5420E26EE66A53C057
:1035F60079F454C07AF4536A546A7B6B0ED0750E14
:103606005324E16E000E5420E26E7BC4E6FF53C0E5
:1036160079F454C07AF4534A542AA4AA79D0A3AAB6
:1036260077D09CA202D09C989C889CA402D0AACF5A
:1036360083F5AACF83F5010E0201765D02E1FF0E46
:10364600755D05E2050183510D0A01E03BD075C2A7
:103656006EF576C26FF5A4BA01D0FDD70501AACFE3
:1036660083F5836B000E851902E1000E841909E1CA
:10367600F70E02017525E16E040E7621E26E83C512
:10368600E6FF000E0501851902E1010E841909E124
:10369600970E02017525E16E040E7621E26E83C552
:1036A600E6FF0201756B766B0501844B852B000ED8
:1036B600851902E1020E841904E1AACF83F5836B12
:1036C600A39A26D0000E851902E1000E841909E19D
:1036D600F70E02017525E16E040E7621E26E83C5B2
:1036E600E6FF000E0501851902E1010E841909E1C4
:1036F600970E02017525E16E040E7621E26E83C5F2
:10370600E6FF020175C26EF576C26FF5754B762B34
:0E3716001AC000F01BC0E1FF1CC0E2FF110052
:1037240000C019F001C018F0156ED8CF16F0E0CF24
:1037340017F0A0A222D0A1A220D0010E3A5C006E04
:10374400000E3B58016E00C03AF001C03BF0150E6C
:103754007B6EA00E7A6E800E006E800E3B18005CAD
:1037640002E13A50000807E3010E0501816F000EE3
:10377400826F7990A092A192A1921750E06E165098
:10378400D86E153A153819C000F018C001F01000B1
:103794000CEC26F0D38CD38AD388D382D3909B6A43
:1037A4009B8CD3B601D0FDD7DDEC10F0640E3A6EDD
:1037B400000E3B6E0601EF99090E896F060E8A6FA3
:1037C400096B05015C6B5D6B000E5D5D02E1280E0B
:1037D4005C5D0AE29C0E5C25E16E060E5D21E26EE4
:1037E400E66A5C4B5D2BF0D75C6B5D6B000E5D5D38
:1037F40002E1800E5C5D0AE2090E5C25E16E060EB4
:103804005D21E26EE66A5C4B5D2BF0D77E86010E8D
:103814007F6E370EB06EAD84B1EC10F00C0E070164
:103824001D6F8CEC05F01F0E0B6E710E0C6E1E0ED0
:103834000D6E0D2EFED70C2EFCD70B2EFAD70000E2
:10384400DF0E0701016F460E026F000E036F47EC97
:103854000EF0D00E0701016F470E026F000E036FCA
:1038640047EC0EF0930E0701016F460E026F000E37
:10387400036F47EC0EF06C0E0701016F480E026FE8
:10388400000E036F47EC0EF03D0E0701016F4A0E68
:10389400026F000E036F47EC0EF0450E0701016F37
:1038A400460E026F000E036F47EC0EF0F70E070191
:1038B400016F480E026F000E036F47EC0EF0F00E1E
:1038C4000701016F450E026F000E036F47EC0EF007
:1038D4009E0E0701016F480E026F000E036F47EC46
:1038E4000EF0CB0E0701016F480E026F000E036F3E
:1038F40047EC0EF0910E0701016F450E026F000EAA
:10390400036F47EC0EF00D0E0B6E2D0E0C6ED70EE2
:103914000D6E0D2EFED70C2EFCD70B2EFAD7000001
:1039240000007C86020E7D6E700EAB6EA884FDECEA
:1039340010F01E0E6E6E89EC11F0E80E0701016F97
:10394400490E026F000E036F47EC0EF0640E3A6EE0
:10395400000E3B6E76EC11F0740E0601DF6F740EF0
:10396400066F100ED26F460E0701016F490E026FEB
:10397400000E036F47EC0EF006C6F2F629EC11F0C8
:1039840000C007F6000E0601086F3CEC0EF0550E61
:103994000701016F4A0E026F000E036F47EC0EF031
:1039A400A4EC0FF000C007F601C008F60A0E0B6E77
:1039B400220E0C6EA10E0D6E0D2EFED70C2EFCD712
:1039C4000B2EFAD794EC11F00A0E0B6E220E0C6E2D
:1039D400A10E0D6E0D2EFED70C2EFCD70B2EFAD792
:1039E400010E0701016F000E026F010E036F000E3E
:1039F400046F1A0E056F4B0E066F000E076F05EC71
:103A04000AF0020E0701016F000E026F010E036F30
:103A1400000E046F090E056F4B0E066F000E076F44
:103A240005EC0AF07A0E0B6EC10E0C6E810E0D6E53
:103A34000D2EFED70C2EFCD70B2EFAD7000000005B
:103A44000D0E2A6E000E2B6EA9DC650E0701016FA8
:103A54004B0E026F000E036F47EC0EF090DC020E6B
:103A64000701016F000E026F010E036F000E046F59
:103A7400920E056F4A0E066F000E076F05EC0AF0F2
:103A84007A0E0B6EC10E0C6E810E0D6E0D2EFED7CE
:103A94000C2EFCD70B2EFAD700000000220E0701D3
:103AA400016F490E026F000E036F47EC0EF0A00E7B
:103AB4000601066FA00EF26F29EC11F000C007F6A4
:103AC400000E0601086F070E0B6E170E0C6E6A0EC1
:103AD4000D6E0D2EFED70C2EFCD70B2EFAD7000040
:103AE400EF9DEF992C6A0501746B756B766B776BA0
:103AF400706B716B726B736B5C6B5D6B000E5D5DF9
:103B040002E17F0E5C5D0BE2860E5C25E16E050E24
:103B14005D21E26E200EE66E5C4B5D2BEFD76B0EE3
:103B24000701016F4A0E026F000E036F47EC0EF09F
:103B340072C5F2F673C5F3F69C0E0601F46F060E19
:103B4400F56F76EC19F09C0EFE6F060EFF6F60ECBD
:103B54000FF0E10E0701016F4B0E026F000E036FB1
:103B640047EC0EF070C5F2F671C5F3F69C0E060133
:103B7400F46F060EF56F76EC19F09C0EFE6F060ED0
:103B8400FF6F60EC0FF03CEC0EF0220E0701016FAA
:103B94004A0E026F000E036F47EC0EF0DFC606F606
:103BA400020E0601FE6F000EFF6F24EC0BF0010EF7
:103BB4000701016F000E026F010E036F000E046F08
:103BC400C50E056F4A0E066F000E076F05EC0AF06E
:103BD4005C0E0B6E510E0C6E600E0D6E0D2EFED72C
:103BE4000C2EFCD70B2EFAD700009D8AA38AF28CE8
:103BF400F28ED08E0501786B796B0D0E2A6E000E55
:103C04002B6ED0EC19F0F0EC19F00D0E2A6E000EAC
:103C14002B6E690E3A6E000E3B6EA8DC0601096B32
:103C2400090E896F060E8A6F9C6B096B090E896FEA
:103C3400060E8A6F89C61DF78AC61EF7A30E0701F2
:103C44001F6F4A0E206F000E216F36EC05F0080E30
:103C540006018925E16E000E8A21E26E62C5E6FF47
:103C6400090E8925E16E000E8A21E26E63C5E6FF26
:103C74000F0E8925E16E000E8A21E26E57C5E6FF1C
:103C8400100E8925E16E000E8A21E26EE66ADFC617
:103C940006F694EC11F0010E0701016F000E026F9D
:103CA400010E036F000E046F89C605F78AC606F776
:103CB40098EC0BF0020E0701016F000E026F010E6B
:103CC400036F000E046FF80E056F4A0E066F000EA8
:103CD400076F05EC0AF0020E0701016F000E026F78
:103CE400070E036F000E046F210E056F000E066FA2
:103CF40098EC0BF01F0E0B6E710E0C6E1E0E0D6EFB
:103D04000D2EFED70C2EFCD70B2EFAD70000000E7A
:103D14000501821902E1000E811907E1000E855D9B
:103D240002E1020E845D01E2F2D7000E851902E180
:103D3400020E841966E19C0E07011D6F060E1E6FAC
:103D4400010E1F6F4C0E206F000E216F36EC05F034
:103D5400F70E0601F26F040EF36F9C0EF46F060E5D
:103D6400F56F070EF66F87EC1AF0000E011802E1EA
:103D7400000E001803E113EC1AF009D0A90E070194
:103D8400016F490E026F000E036F47EC0EF09C0E9C
:103D940007011D6F060E1E6FF90E1F6F4B0E206F6D
:103DA400000E216F36EC05F0970E0601F26F040E3B
:103DB400F36F9C0EF46F060EF56F070EF66F87EC2B
:103DC4001AF0000E011802E1000E001811E106ECD1
:103DD40014F000C035F001C036F0000E011802E105
:103DE4000A0E001804E1BEEC11F0F8EC15F009D04D
:103DF400690E0701016F490E026F000E036F47EC55
:103E04000EF081A20BD12C50000AD8A407D10501D1
:103E140057510008D8B002D1240E07011D6F8CEC55
:103E240005F0090E07011D6F8CEC05F0800E0701EB
:103E3400016F4A0E026F000E036F47EC0EF072C55D
:103E4400F2F673C5F3F69C0E0601F46F060EF56FD9
:103E540076EC19F09C0EFE6F060EFF6F60EC0FF00F
:103E6400F10E0701016F4B0E026F000E036F47EC5A
:103E74000EF070C5F2F671C5F3F69C0E0601F46FF0
:103E8400060EF56F76EC19F09C0EFE6F060EFF6FB2
:103E940060EC0FF03CEC0EF00601EFB90ED0EF8DA4
:103EA4008D880501706B716B726B736B746B756BC2
:103EB400766B776B0601EF892C6A05017351030851
:103EC40002E17251FE0823E20601EF9D81A21FD098
:103ED4008D98100E0B6E390E0C6E0D0E0D6E0D2E90
:103EE400FED70C2EFCD70B2EFAD7000000008D88CD
:103EF400100E0B6E390E0C6E0D0E0D6E0D2EFED7C0
:103F04000C2EFCD70B2EFAD700000000DFD70601D9
:103F1400EFAD84D0050157513008D8B07FD0000EE2
:103F2400711902E1000E701944E18D88000E7319B5
:103F340002E1000E721929E1860E0701016F050ED8
:103F4400026F210E036F000E046F080E056F000E42
:103F5400066FDDEC09F005018F6BA60E0701016FFA
:103F6400050E026F440E036F000E046F090E056FF9
:103F7400000E066FDDEC09F00501B06BFF0E0601C3
:103F8400F26F030EF36F6AEC18F005015C6B5D6B66
:103F9400000E5D5D02E1800E5C5D0BE2860E5C2529
:103FA400E16E050E5D21E26E200EE66E5C4B5D2B2C
:103FB400EFD7050E026E70C500F071C501F0025016
:103FC40005E0003600900136FF0FFAD7860E002474
:103FD4000701016F050E0120026F550E036F000EDD
:103FE400046F200E056F000E066FDDEC09F005016D
:103FF400704B712B000E006E7151005C02E1705128
:1040040003080CE272C5F2F673C5F3F66AEC18F015
:104014000501724B732B706B716B8D9881B276D0E6
:104024000601EFAD69D0890E0701016F490E026FD9
:10403400000E036F47EC0EF00601EF9DEF998D988B
:104044000501706B716BFF0E0601F26F030EF36FC7
:10405400E0EC18F0C90E0701016F490E026F000E63
:10406400036F47EC0EF0400E05015C6F000E5D6FB0
:10407400000E5D5D02E1800E5C5D0BE2860E5C2548
:10408400E16E050E5D21E26E200EE66E5C4B5D2B4B
:10409400EFD7C60E0701016F050E026F210E036FE5
:1040A400000E046F090E056F000E066FDDEC09F0BB
:1040B400E60E016F050E026F440E036F000E046FCF
:1040C4000A0E056F000E066FDDEC09F0FF0E060107
:1040D400F26F030EF36F6AEC18F0080E0701016F1C
:1040E400480E026F000E036F47EC0EF00501706B73
:1040F400716B010E2C6E0AD08DB802D08C9801D051
:104104008C888CB802D08D8801D08D982C50010AEF
:10411400D8A4F5D087B6F3D05C0E0701016F470E23
:10412400026F000E036F47EC0EF087B601D0FDD787
:104134003D0E0B6EE10E0C6E3F0E0D6E0D2EFED776
:104144000C2EFCD70B2EFAD70000000087A601D056
:10415400FDD7060E0701016F4A0E026F000E036FB2
:1041640047EC0EF072C5F2F673C5F3F69C0E060129
:10417400F46F060EF56F76EC19F09C0EFE6F060ECA
:10418400FF6F60EC0FF03CEC0EF0FF0E0601F26FD7
:10419400030EF36FE0EC18F089C61DF78AC61EF70C
:1041A400BE0E07011F6F4B0E206F000E216F36EC01
:1041B40005F089C601F78AC602F7860E0701036F68
:1041C400050E046F30EC0FF089C601F78AC602F7BA
:1041D400370E036F000E046F30EC0FF089C601F741
:1041E4008AC602F7A60E036F050E046F30EC0FF0BB
:1041F40089C6FEF68AC6FFF660EC0FF03CEC0EF0C2
:1042040089C61DF78AC61EF7090E07011F6F4C0EDB
:10421400206F000E216F36EC05F089C601F78AC6BF
:1042240002F7C60E0701036F050E046F30EC0FF0A2
:1042340089C601F78AC602F7320E036F000E046FB7
:1042440030EC0FF00601056B89C601F78AC602F748
:10425400E60E0701036F050E046F30EC0FF089C6FC
:10426400FEF68AC6FFF660EC0FF03CEC0EF03CEC78
:104274000EF0FA0E0701016F430E026F000E036F7A
:1042840047EC0EF005015C6B5D6B73515D5D02E103
:1042940072515C5D10E25CC5F2F65DC5F3F6E0ECCC
:1042A40018F0860EFE6F050EFF6F60EC0FF005012F
:1042B4005C4B5D2BEAD71F0E0701016F470E026F9F
:1042C400000E036F47EC0EF0960E0701016F470EC8
:1042D400026F000E036F47EC0EF03D0E0B6EE10E05
:1042E4000C6E3F0E0D6E0D2EFED70C2EFCD70B2E32
:1042F400FAD70000000087A601D0FDD72C6A000E73
:104304000401781902E1010E771971E1F0EC19F05A
:10431400570E0701016F4B0E026F000E036F47EC3F
:104324000EF0750E0601FE6F000EFF6F60EC0FF0CD
:104334003CEC0EF0DFC606F694EC11F09C0E060180
:10434400F26F060EF36F750EF46F000EF56F100E1C
:10435400F66F000EF76FB4EC15F0010E0701016F54
:10436400000E026F010E036F000E046F3B0E056F0B
:104374004B0E066F000E076F05EC0AF0020E0701E4
:10438400016F000E026F010E036F000E046F9C0E8E
:10439400056F060E066F98EC0BF03D0E0B6EE10EEA
:1043A4000C6E3F0E0D6E0D2EFED70C2EFCD70B2E71
:1043B400FAD700000000750E0601F26F000EF36FCD
:1043C4002D0EF46F000EF56F040EF66F87EC1AF0E5
:1043D400000E011802E1000E001807E1790E060133
:1043E400F26F000EF36FA3EC11F0D0EC19F0F0ECC7
:0643F40019F00FD4FFD701
:104C180010EE1DF0320E006E010E016E3A0EF66EA9
:0E4C2800480EF76E000EF86EF5EC10F012005C
:1043FA003C3F786D6C2076657273696F6E3D223131
:10440A002E302220656E636F64696E673D225554B3
:10441A00462D38223F3E0D3C6B6D6C20786D6C6EDC
:10442A00733D22687474703A2F2F7777772E6F70E6
:10443A00656E6769732E6E65742F6B6D6C2F322EE5
:10444A0032223E0D3C446F63756D656E743E0D3CC1
:10445A005374796C652069643D22707572706C655D
:10446A00506F6C79223E0D3C4C696E655374796CC1
:10447A00653E0D3C636F6C6F723E37666666303020
:10448A0066663C2F636F6C6F723E0D3C776964748D
:10449A00683E343C2F77696474683E0D3C2F4C6942
:1044AA006E655374796C653E0D3C506F6C7953742C
:1044BA00796C653E0D3C636F6C6F723E37663030C7
:1044CA00666630303C2F636F6C6F723E0D3C2F5026
:1044DA006F6C795374796C653E0D3C2F5374796C0B
:1044EA00653E0D3C506C6163656D61726B3E3C7359
:1044FA0074796C6555726C3E23707572706C655078
:10450A006F6C793C2F7374796C6555726C3E0D3CF7
:10451A004C696E65537472696E673E0D3C657874BA
:10452A00727564653E313C2F657874727564653EB8
:10453A000D3C74657373656C6174653E313C2F7410
:10454A00657373656C6174653E0D3C616C74697466
:10455A007564654D6F64653E6175206E6976656147
:10456A007520647520736F6C3C2F616C7469747567
:10457A0064654D6F64653E0D3C636F6F7264696E6E
:07458A00617465733E0D0032
:1045910020626F75746F6E2042503220285248336A
:1045A10029206465206C6120636172746520636CED
:1045B10069636B65722020706F75722076616C691A
:1045C100646572206C612043617074757265206648
:1045D100696368696572204B4D4C2067E96E72E929
:0F45E1002073757220646973706C61790D0A0024
:1045F0002055415254322031393230302C382C4E33
:104600002C3120436C69636B657232204D696B728B
:104610006F4275732331205247312C524732203C70
:104620002D3E204750532055424C4F5820374E289E
:10463000362050696E732955415254202B20616CED
:05464000696D0D0A0088
:104645002055415254312033383430302C382C4EDB
:104655002C3120436C69636B657232204D696B7236
:104665006F6275732332205243362C524337203CF8
:104675002D20504C32333033202D203E7465726D21
:0E468500696E616C205642524159200D0A00A8
:1046930020536F75726365204D696B726F432043BE
:1046A3006C69636B6572325F31384638374A35302F
:1046B3005F4750535F55424C4F585F374E5F7365AA
:1046C300756C5F4C43445F454570726F6D314D426D
:0C46D3005F3136303931332E630D0A00A0
:1046DF002048617264776172653A200D0A20436C3D
:1046EF0069636B6572322031384638374A3530206E
:1046FF005375727669766F72202B204750532D4376
:10470F004F4D5053202055426F7820374E0D0A00E1
:10471F003C2F636F6F7264696E617465733E0D3CFD
:10472F002F4C696E65537472696E673E3C2F506CE7
:10473F006163656D61726B3E0D3C2F446F63756DE8
:0D474F00656E743E3C2F6B6D6C3E200D00BE
:10475C000D0A436C65617220427566666572207441
:10476C0065726D696E616C20646973706C6179201F
:10477C00210D0A2045742061707075796572207363
:0A478C007572204250320D0A200021
:104796000D0A0D0A20526563757065726572206C8C
:1047A600652066696368696572204B4D4C20210D52
:1047B6000A20457420617070757965722073757270
:0A47C600204250320D0A0D0A2000B7
:1047D000204469726563746F7279203A20433A5FAE
:1047E0004D696B726F435F4D657350726F6A65748C
:1047F000735F4D696B726F435F31384638374A35A6
:08480000305F4750530D0A0020
:10480800417070757965722073757220425032203C
:10481800706F757220726563757065726572206C51
:1048280065206C697374696E67204B4D4C2E2E0D94
:024838000A0074
:02483A002C0050
:02483C002C004E
:09483E0030312F30312F313600EA
:024847000D0062
:01484900006E
:05484A004364653D0020
:03484F0020200026
:02485200000064
:0348540020200021
:024857006400FB
:04485900000000005B
:02485D00200039
:02485F00200037
:0B48610030304830304D303053200024
:10486C0020464F53433D384D687A20696E7465720B
:10487C006E65207820504C4C203D3E2034384D68DD
:10488C007A2020416C696D203A20332C3356200D50
:02489C000A0010
:10489E00204465636F64616765206465203220542F
:1048AE0072616D6573204E4D45413A202047504749
:0D48BE004741202B204750524D430D0A006A
:1048CB0020436F6D6D75746174657572202852424B
:1048DB0031292053746F72655F4461746173207367
:0C48EB00757220454570726F6D0D0A005B
:1048F700204C696169736F6E20504943203C2D3EFF
:1049070020204D6F64756C65204750532055424CED
:0B4917004F5820374E2020200D0A00D2
:10492200436865636B2070726573656E63652032E0
:104932003446433130323620617420402030784191
:04494200340D0A0026
:10494600436865636B2070726573656E6365204CA2
:104956004344323131392061742040203078373475
:034966000D0A0037
:1049690042414420526563657074696F6E206F75AA
:10497900204465636F64616765204747410D0A00FC
:104989000D0A46696E2064652073746F636B6167F5
:1049990065207375722032344643202E2E0D0A008D
:1049A90042414420526563657074696F6E206F756A
:1049B900204465636F6461676520524D430D0A00A9
:1049C9005465726D696E6520656372697475726587
:0F49D900207375722032344643202E2E0D0A00B3
:1049E8000D0A496E69742049324332204861726465
:0E49F80077617265203430304B687A0D0A000A
:104A06000D0A4E756D506167652066696E616C2092
:0C4A160032344C4331303236203D200059
:104A2200200D0A41726D652049542055415254317E
:0B4A320020262055415254320D0A008E
:104A3D00204C696169736F6E20504943203C2D3EB7
:084A4D002050433A200D0A003D
:104A550020496E6974204C4344203231313920326B
:064A65007831360D0A0055
:104A6B002032344C433130323620204E756D50613C
:054A7B0067653D20000D
:104A80000D0A204E756D506167652032344C433DF0
:024A9000200004
:104A9200496E697420414443207375722045413147
:014AA2000013
:104AA3004E62205361743A202020204669783A20D0
:014AB3000002
:104AB4004C4F4E3A2020202020202020202020204F
:014AC40000F1
:104AC50041726D6520496E746572727570747320DC
:014AD50000E0
:104AD6004C41543A20202020202020202020202035
:014AE60000CF
:104AE700416C74697475643A2020202020202020AE
:014AF70000BE
:104AF80044617465203A2020202020202020202096
:014B080000AC
:104B0900203130302078203430203D2034736563E3
:014B1900009B
:104B1A00496E69742054696D6572332034306D535F
:014B2A00008A
:104B2B00436865636B2044657669636520402000AC
:0E4B3B0055415254312052656375203A2000D6
:0E4B4900206973206E6F7420666F756E6400B5
:0E4B570055415254312052656375203A2000BA
:0D4B650020496E697420414443310D0A005F
:0C4B720020204820204D2020532020004F
:0C4B7E002020202020416C74203A2000F0
:0C4B8A002020202048444F50203A2000FA
:0B4B9600202020536174656C3A200061
:0A4BA100202020204669783A200009
:0A4BAB0020666F756E64204F4B000A
:094BB5004A4A2F4D4D2F414100E9
:094BBE004465627574203A200080
:094BC70020204C6174203A20000A
:094BD000322020484152445700F4
:084BD900206F6E2049324300F9
:084BE10020496478203D20000A
:084BE900204C6F6E203A200001
:084BF10020204964783D2000FA
:084BF9002447504747412C00FE
:084C0100244750524D432C00E2
:074C090046696E203A20000D
:074C10004C54433A20200040
:020000040001F9
:06FFF800ACF7C5FFF8FFA5
:00000001FF
